:1000000000308A009C290000FF00030E8301A60037
:100010007F08A5000A08AD008A01A50E0408A70004
:100020002008A8002108A9002208AA002308AB0084
:100030002408AC00831383128C308400801D222896
:100040008C193528270884002808A0002908A10059
:100050002A08A2002B08A3002C08A4002D088A005F
:10006000260E8300FF0E7F0E09008A115F280A10FA
:100070008A100A1182070D340A3449343234433469
:10008000203453346C346134763465342034533442
:1000900074346134723474346534643421340D340E
:1000A0000A34003413084408930014168C11831684
:1000B000141858288312A101141AA10A00348316B7
:1000C000941A67288312BF011318BF17831683126F
:1000D0003F08BF0AB0003E1430087F3C031C98283C
:1000E000B008031D7328300B7E288316141C762855
:1000F00083121308AF002F08B100BE143008023C71
:10010000031D8B288316141C832883121308AF0049
:100110002F08B2003E153008033C031D98288316B3
:10012000141C902883121308AF002F08B300BE15CB
:100130003008803C031DA5283108C4005220320835
:10014000C40052203308C40052208C118A11222886
:1001500040308400831300080319BC280130A1003B
:10016000A001A00BB128A10BB0284A30A000A00B21
:10017000B728BA28800BAE280034B5013308B40084
:100180003408B500B4013208B4070318B50A310BBE
:10019000D828340BD328B508031DD328831607119C
:1001A00083120715D72883160711831207111B29FD
:1001B00031080A3C031DFA283508B7003408B60098
:1001C0003708063C0318EF28FF3A031DEB283608D2
:1001D000083C0318EF280730B7000830B60036088F
:1001E000083CB8000730B9003708031C370FB902C4
:1001F0003E161B293108143C031D1B293508BB0082
:100200003408BA003B08063C03181129FF3A031DC5
:100210000D293A08083C031811290730BB000830A3
:10022000BA003A08083CBC000730BD003B08031C7C
:100230003B0FBD02BE163E10BE103E11BE118A110C
:10024000FE291230C102031C34294130840083137B
:10025000FC3080050310800C800C00080319342941
:1002600032290000800B312900343E1E5E2983169E
:10027000071083120714A630A000A00B3D29000030
:100280003708C000C00AC00303194A29FF30C10063
:10029000212143293608C10021218316071083122A
:1002A00007103908C000C00AC00303195B29FF30DA
:1002B000C100212154293808C1002121BE1E8729EF
:1002C0008316871083128714A630A000A00B66291E
:1002D00000003B08C000C00AC00303197329FF30A7
:1002E000C10021216C293A08C10021218316871001
:1002F000831287103D08C000C00AC0030319842977
:10030000FF30C10021217D293C08C10021213E1E72
:100310008F29BE1E8F291030C000A8209A293E1AAE
:100320009729BE1A97291430C000A8209A291230A4
:10033000C000A8208A11FF29840183131F30830580
:100340008316061706161030930036308312940079
:1003500083169B1119309900A630980090308312B3
:10036000980003171F109F101F119F1103131F13D5
:10037000003003179E0099019A0183169E01831293
:100380009B0103138D12AE010330BF00C830C000C3
:10039000A820031799019A0183169E0183129B01DD
:1003A00003138D1203179801FF3083160313850082
:1003B0007F3086005C3087008312C0014008372000
:1003C000C00AA00020080C1EE32999001630400244
:1003D000031DDE293E10BE103E11BE113E123E121C
:1003E00083168C15C03083128B043E1CFE29BE1C64
:1003F000FE293E1DFE29BE1DFE29BD283529F529F1
:02040000630097
:02400E00E23F8F
:00000001FF
